:1007F4000000000000000000FF00FF00FF00FF00F9
:10080400AAAAAAAAAAAAAAAAAAF0F0F0F00F0F0FFD
:100814000FF03FF03FF03FF03FF08040201008041D
:100824000201FFFFFFFFFFFFFFFFFF0000000000CA
:1008340000000000000000000000000000000000B4
:1008440000000000000000000000000FFC1F8E4F9D
:10085400F8FC00103F8FFFFFFF81F2FC7E000000D8
:10086400FC0FFFFFC00000000003070619C30C3093
:1008740000300E02631981830E3018000000300C22
:100884006330700000000003038630C30630003874
:1008940006044309808406301800000030086130E3
:1008A400380000000003018630430630005803047A
:1008B4000301800C0630180000003000603018007E
:1008C4000000000300C638430630004C01880301D1
:1008D4008218023018000000300060300C00000064
:1008E400000300C61C030630004C0190030182186B
:1008F400003018000000300060300C0000000003DD
:1009040000C60F030C30008C00D00301FE18003F1A
:10091400F8000000300060300C000000000300C646
:100924000383F83000860060030182180030180049
:100934000000300060300C000000000300C601C35A
:10094400003001FE0060030182180030180000002E
:10095400300060300C000000000300C620E30030CB
:100964000106006003018018003018000000300008
:1009740060300C0000000003018620630030120385
:1009840000600301804C0230180000003010603019
:1009940018000000000303063063003032030060D7
:1009A4000301808C043018000000303060303000C7
:1009B40000000003060638C30030660380600301AC
:1009C400818708301800000030606030600000004B
:1009D400000FFC1FA78FC0FFEF07C1F80FC7FF81EF
:1009E400F0FC7E000000FFE1F8FFC0000000000002
:1009F40000000000000000000000000000000000F3
:0B0A04000000000000000000000000E7
:040003008E098F0AC9
:10000700E4FFFEC3EF950AEE9509503BE4FDFCC300
:10001700ED9405EC9400502820A01EE4FBFAC3EBF6
:1000270094A8EA946150070BEB70010A80F020A0B6
:10003700FDAE09AF0A7C007D050DED70010C80CF88
:070047000FEF70010E80BCF9
:01004E00228F
:10004F00E4FDFCC3ED9FEC9E501AE4FBFAC3EB9466
:10005F0005EA940050070BEB70010A80F00DED706C
:04006F00010C80DF21
:01007300226A
:10007400E4FDFCC3ED9FEC9E50070DED70010C8078
:01008400F289
:010085002258
:10008600A2009290D2928F807F017E00120074C2ED
:0400960091D2912250
:10009A00AB07D2927F15C200120086AF08D20012B7
:1000AA0000867F50D2001200867F5CC20012008652
:1000BA00D290E4FFFEC3EF9403EE9400501FAD0309
:1000CA00530580ED60057580FF8003E4F580C291D9
:0F00DA00D291EB25E0FB0FEF70010E80D80508E7
:0100E90022F4
:1000EA00D290D292E4FDFCC3ED9408EC9400501F28
:1000FA00AE07530680EE60057580FF8003E4F58045
:10010A00C291D291EF25E0FF0DED70010C80D87FEE
:06011A00057E00120074D6
:0101200022BC
:100121008F13D2927F15C200120086AF08D200123F
:1001310000867F50D2001200867F5CC200120086CA
:10014100D290E4FBFAC3EB9403EA94005021A91383
:10015100530180E960057580FF8003E4F580C29159
:10016100D291E51325E0F5130BEB70010A80D6055A
:10017100087F15C200120086AF08D2001200867FE8
:1001810050D2001200867F5CC200120086D290E439
:10019100FAFBC3EB9403EA94005021A913530180A5
:1001A100E960057580FF8003E4F580C291D291E595
:0E01B1001325E0F5130BEB70010A80D605084C
:0101BF00221D
:1001C000C2947FE87E0312004FC2937F647E0012C8
:1001D000004FD2937FE87E0312004F7F30C200129F
:1001E00000867F94C2001200867FD1C20012008672
:1001F0007F20C2001200867F08D20012008674F4AD
:10020000FF7E0112004F7F20C2001200867F0BD2BA
:10021000001200867F81C2001200867F18D2001271
:1002200000867F04D2001200867FCAC200120086B8
:10023000E4FFD2001200867F23D200120086E4FF82
:10024000D2001200867FA7C2001200867FBBC200C8
:100250001200867F02D2001200867FBCC20012000C
:1002600086E4FFD200120086E4FFD2001200867FEF
:1002700004D2001200867F75C200120086E4FFD20D
:10028000001200867F9FD2001200867F15C20012E6
:1002900000867F15D2001200867F54D2001200869D
:1002A0007FA9C2001200867F31C2001200867F3211
:1002B000C2001200867F01D200120086E4FFD20045
:1002C0001200867F02D2001200867F34C200120024
:1002D000867F20C200120086E4FFD2001200867FD3
:1002E00002D2001200867F04D2001200867F06D25E
:1002F000001200867F08D2001200867F0AD2001208
:1003000000867F0CD2001200867F0ED2001200867B
:100310007F10D2001200867F12D2001200867F1456
:10032000D2001200867F16D2001200867F18D200FB
:100330001200867F1AD2001200867F1CD2001200A3
:10034000867F1FD2001200867F21C200120086E441
:10035000FFD2001200867F02D2001200867F04D2F4
:10036000001200867F06D2001200867F08D200129B
:1003700000867F0AD2001200867F0CD2001200860F
:100380007F0ED2001200867F10D2001200867F12EC
:10039000D2001200867F14D2001200867F16D2008F
:1003A0001200867F18D2001200867F1AD200120037
:1003B000867F1CD2001200867F1FD2001200867F2B
:1003C00030C2001200867FAFC2001200867F647EBA
:0503D0000012004F22A5
:0603D5008B098A0A890B66
:1003DB00751210E4F5087F75C2001200867F10D2EB
:1003EB00001200867F10D200120086E4F50CF50D8A
:1003FB00C3E50D9440E50C9400506BE4F50EF50F3E
:10040B00C3E50F9401E50E94005051E4F510F5117E
:10041B00C3E5119428E5109400501DAB09AA0AA955
:10042B000B850F82850E83120A1BFF12012105110A
:10043B00E5117002051080D80512E4F5087F75C22E
:10044B0000120086AF12D200120086AF12D2001239
:10045B000086050FE50F7002050E80A4050DE50D56
:10046B007002050C808A751250E4F5087F75C20086
:10047B001200867F50D2001200867F50D2001200ED
:10048B0086E4F50CF50DC3E50D9440E50C94005096
:10049B006BE4F50EF50FC3E50F9401E50E940050D8
:1004AB0051E4F510F511C3E5119428E510940050B3
:1004BB001DAB09AA0AA90B850F82850E83120A1B95
:1004CB00FF1201210511E5117002051080D80512EC
:1004DB00E4F5087F75C200120086AF12D20012003D
:1004EB0086AF12D200120086050FE50F7002050EC3
:0C04FB0080A4050DE50D7002050C808A40
:0105070022D1
:100508007A10E4F5087F75C200120086AF02D200A7
:10051800120086AF02D200120086E4F509F50AC37C
:10052800E50A9450E5099400500F7FFF12009A05E0
:100538000AE50A7002050980E60AE4F509F50AC326
:10054800E50A943FE5099400504C7F75C2001200FB
:1005580086AF02D200120086AF02D200120086E4F3
:10056800F5087F8012009AE4F50BF50CC3E50C94AE
:100578004EE50B9400500FE4FF12009A050CE50CB1
:100588007002050B80E67F2012009A0A050AE50A28
:100598007002050980A97A50E4F509F50AC3E50A4D
:1005A800943FE5099400504C7F75C200120086AF55
:1005B80002D200120086AF02D200120086E4F508CB
:1005C8007F8012009AE4F50BF50CC3E50C944EE518
:1005D8000B9400500FE4FF12009A050CE50C700212
:1005E800050B80E67F2012009A0A050AE50A7002C8
:1005F800050980A97F75C200120086AF02D20012D9
:100608000086AF02D200120086E4F508F509F50A63
:10061800C3E50A9450E5099400500F7FFF12009A31
:0A062800050AE50A7002050980E6E4
:0106320022A5
:060633008B098A0A890B05
:10063900751610E4F510F511F512F513C3E51394C9
:1006490004E512940040030206E4E4F510F511F5FF
:100659000CF50DC3E50D9410E50C940050727F75EF
:10066900C200120086AF16D200120086AF16D20061
:100679001200867F15C200120086E4FFD200120024
:10068900867F50D2001200867F5CC200120086E489
:10069900F50EF50FC3E50F941EE50E94005025AB3A
:1006A90009AA0AA90B851182851083120A1BFF1258
:1006B90000EA0511E51170020510050FE50F70023A
:1006C900050E80D00516050DE50D7002050C808319
:1006D9000513E51370020512020645751650E4F577
:1006E90012F513C3E5139404E512940040030207BD
:1006F9008BE4F510F511F50CF50DC3E50D9410E536
:100709000C940050727F75C200120086AF16D20099
:10071900120086AF16D2001200867F15C2001200A1
:1007290086E4FFD2001200867F50D2001200867F35
:100739005CC200120086E4F50EF50FC3E50F941EA6
:10074900E50E94005025AB09AA0AA90B85118285EB
:100759001083120A1BFF1200EA0511E51170020548
:1007690010050FE50F7002050E80D00516050DE581
:100779000D7002050C80830513E513700205120242
:0207890006EC7C
:01078B00224B
:10078C001201C01201C07B057A0779F41203D57BE4
:10079C00057A0879261203D57F887E1312004F7FC5
:1007AC00987E3A1200031205087F887E1312004FC0
:1007BC007F987E3A1200037B057A0879041203D5E0
:1007CC007F887E1312004F7F987E3A1200037B05C0
:1007DC007A08792F1206337F887E1312004F7FA878
:0807EC007E61120003809C22D3
:03000000020A0FE2
:0C0A0F00787FE4F6D8FD75812002078C8A
:100A1B00BB020CE58229F582E5833AF583E022409F
:100A2B0003BB0406E92582F8E622400DE58229F591
:0F0A3B0082E5833AF583E49322E92582F8E222EB
:00000001FF
